:100000002BC043C042C041C040C03FC09FC03DC0A4
:100010003CC03BC03AC04D0020002000204D487A33
:1000200000204D002020200020504C4C2053594EE1
:100030005448455349530A002076312E30206279C6
:1000400020447573616E0020202020202020202075
:10005000202020202020200011241FBECFEDCDBF66
:1000600010E0A0E6B0E0E8EBF7E003C0C8953196F9
:100070000D92AE36B107D1F710E0AEE6B0E001C0A8
:100080001D92AE37B107E1F7BAC1BACF8DE382BF97
:1000900085E083BF89B7826089BF0895B898BE9A0A
:1000A0008FE181BBC69808951F93CF93DF93D92F1B
:1000B000C82F9498939A929A81E090E034D09298C5
:1000C00010E0D7FF02C0949A01C09498929A81E000
:1000D00090E029D09298CC0FDD1F1F5F103188F37C
:1000E00093988AE090E004D0DF91CF911F9108951A
:1000F000CF93DF93181619064CF4D92FC82F929A74
:1001000081E090E010D092982197C9F7DF91CF91CC
:10011000089584E190E0ECDF80E09CECC5DF80E0B6
:100120009CECC2DF089540E050E04817590768F49E
:1001300030E020E0275E2A3FE8F33F5F3634C8F323
:100140004F5F5F4F4817590798F3089578941F92AF
:100150000F920FB60F9211241F932F933F934F933B
:100160005F936F937F938F939F93AF93BF93CF933F
:10017000EF93FF93B09906C080916E008F5F8093DC
:100180006E0002C010926E00859906C080916F00CB
:100190008F5F80936F0002C010926F00869906C037
:1001A000809170008F5F8093700002C01092700089
:1001B00080917100882309F444C080916E008130E1
:1001C00029F4809173008F5F8093730080916F009A
:1001D000813029F480917300815080937300809165
:1001E0007300853018F084E080937300C091700034
:1001F000CC2319F482E080937100C130A1F4809186
:100200007100823081F4809173009927880F991FC3
:1002100060917C0070917D0094D2109271001092D8
:100220007200C093740061E08CE074D186E190E0CC
:1002300038D280917B008A3008F4BBC088E190E01E
:10024000C1C0C0917000CC23D9F41091720011305C
:10025000B9F4809173008F5F80937300853010F044
:10026000C0937300809173009927880F991F5CD207
:1002700090937D0080937C00C09372001093740073
:1002800050917000513011F450937200543128F0A5
:1002900081E08093710010927B0060916E0061306C
:1002A00059F480917C0090917D00059690937D009B
:1002B00080937C0010927400643158F080917C002F
:1002C00090917D000A9690937D0080937C0010921F
:1002D000740040916F00413059F480917C009091FE
:1002E0007D00059790937D0080937C0010927400B0
:1002F000443158F080917C0090917D000A97909352
:100300007D0080937C001092740080917C0090911D
:100310007D008056924244F480E692E290937D0004
:1003200080937C001092740080917C0090917D00FD
:1003300081539A4244F080E39AE290937D00809347
:100340007C00109274008091790090917A00209145
:100350007C0030917D008217930769F0552359F492
:10036000662349F4442339F430937A0020937900CA
:10037000932F822F99DE61E0862FCCD080917C0074
:1003800090917D00805197421CF48AE190E089D1E0
:100390004FEF62E080917C0090917D00F7D08CE17E
:1003A00090E07FD180917400882351F081E290E049
:1003B00078D18091730099274FEF60E0E7D003C0B8
:1003C00084E290E06ED180917B008F5F80937B0010
:1003D000843111F410927B00FF91EF91CF91BF9186
:1003E000AF919F918F917F916F915F914F913F91CD
:1003F0002F911F910F900FBE0F901F901895CFED6A
:10040000D0E0DEBFCDBF42DE49DE83DE60D181E0D9
:100410006FD060E0862F7ED088E290E042D188E302
:1004200090E03FD180ED97E07EDE809173009927C8
:10043000880F991F79D190937D0080937C0081E093
:100440008093740010927300682F80E063D087E47B
:1004500090E027D17894FFCF611571058105910552
:1004600029F06150704080409040D9F708951F9363
:10047000CF93C82F162F80917600882309F427D1B7
:10048000C498C398C298C198C798113009F4C79A04
:100490002C2F332724FDC49A25FDC39A26FDC29A2A
:1004A000C7FDC19AC59891E09A95F1F7C59A91E078
:1004B0009A95F1F7C498C398C298C198123081F008
:1004C00020FDC49A21FDC39A22FDC29A23FDC19A40
:1004D000C59891E09A95F1F7C59A91E09A95F1F750
:1004E0006FE370E080E090E0B7DFCF911F91089557
:1004F0001F93182F60E0BBDF1150123048F468EDF5
:1005000079E080E090E0A8DF109277001092780008
:100510001F9108951F93CF93C82F162F1092750027
:10052000803110F4623020F081E0809375000CC0BF
:10053000E62FFF27E05AFF4F80818C0F8058D8DFCD
:10054000C093770010937800CF911F910895982F52
:10055000809175008823C1F49A3051F4909178000D
:10056000992391F4892F8F5F682F892FD3DF089506
:1005700080917700803140F461E0892F78DF8091AD
:1005800077008F5F8093770008950895DF92EF9250
:10059000FF920F931F93CF93DF93CDB7DEB72997C9
:1005A0000FB6F894DEBF0FBECDBF082F192FE62E71
:1005B00089E0AC2FBD2F1196E4E6F0E001900D929A
:1005C0008A95E1F7DD2499E0F92E17FF07C0109511
:1005D00001951F4F8DE2898381E0D82EEE2089F0AE
:1005E00089E090E08F1991092E2D33278217930708
:1005F00040F0FA94FD2FEC2FEF0DF11D8EE2818378
:10060000EE24FA942C2F3D2F2F5F3F4FF32FE22F34
:10061000EF0DF11D912F802F6AE070E0A4D0805D76
:100620008083912F802F6AE070E09DD0062F172FD6
:10063000672B11F4EE2019F085E08E1578F61D2D4C
:1006400088E08F1588F0B32FA22FA10FB11DF32FD3
:10065000E22FEF0DF11D80818C9380E280831F5F7C
:10066000F39488E08F1578F7493008F4142FFF24AD
:10067000F11648F4FD2FEC2FEF0DF11D818167DF9E
:10068000F394F116B8F329960FB6F894DEBF0FBEB7
:10069000CDBFDF91CF911F910F91FF90EF90DF9031
:1006A0000895CF93DF93D92FC82FF92FE82F2196E4
:1006B000C895802D882341F04ADFFD2FEC2F21962D
:1006C000C895802D8823C1F7DF91CF9108951F939E
:1006D00011E010937600BD9AC59ABF9ABC9ABB9A56
:1006E000BA9AB99A61E172E880E090E0B5DE62E022
:1006F00080E3BDDE61E07AE180E090E0ADDE62E0C3
:1007000080E3B5DE62E080E3B2DE62E080E2AFDE8D
:1007100088E2EEDE88E0ECDE812FEADE86E0E8DECD
:100720008CE0E6DE1F910895E199FECF9FBB8EBB62
:10073000E09A01960DB29FBB8EBBE09A802D9DB3CF
:100740000895FFEF0FB6E199FECF9FBB8EBB6DBB47
:10075000F894E29AE19A0FBEF0FF08958F5F9F4FE1
:10076000672FFF27F0CF97FB092E07260AD077FDCA
:1007700004D00CD006D000201AF4709561957F4FFC
:100780000895F6F7909581959F4F0895AA1BBB1B7E
:1007900051E107C0AA1FBB1FA617B70710F0A61B81
:1007A000B70B881F991F5A95A9F780959095682FC8
:0807B000792F8A2F9B2F089579
:0E07B80000401454202020202020202020006B
:00000001FF
